:1000000000308A0004280000FF238316900000308F
:100010008A0083129F280A108A100A11820700346E
:10002000FE34FD34FB34F734EF34DF34BF347F3437
:10003000FE340A108A100A1182070034F934A434FD
:10004000B034993492348234F83480349834C034E3
:100050000A30B5003208B3003108B4000130B600F0
:100060003608103C031C4D280314B30DB40D0318BF
:100070003B2805103C2805140630A000A00B3E28A4
:10008000000005150330A000A00B44280511033023
:10009000A000A00B4928B60A3028051000342F30E4
:1000A00084000008031963280130A100A001A00BFF
:1000B0005728A10B56284A30A000A00B5D2800004D
:1000C0000000800B542800346430AC000130AD00D7
:1000D0002D08093C031C81282D080B20AF002B089C
:1000E0001920B0002F08B1003008B2002820643079
:1000F000AF004F20851485102C08AF004F20AD0AAB
:100100006828AD012D08083C031C9E282D08083CDA
:10011000AE002E080B20AF002B081920B0002F08CE
:10012000B1003008B20028206430AF004F208514A1
:1001300085102C08AF004F20AD0A822801298401C8
:100140001F30830507309F00A401A601A901AA0161
:1001500000306500073099008316050803308312CC
:10016000A000A00BB12819088C110130A5002408AB
:10017000FB3E0318DA28053E1229FF30A700FF30A6
:10018000A8000A30A900DA28A701FF30A800A901B9
:100190000A30AA00DA280130A9000930AA00DA28BA
:1001A0000230A9000830AA00DA280630A90004307D
:1001B000AA00DA28A3012308C83C031CF6288510EE
:1001C0002708B1002708B2002820851485102908C7
:1001D000AF004F202808B1002808B200282085145D
:1001E00085102A08AF004F20A30ADB28A40A2408A0
:1001F000043C0318B7280230AF004F202508AB009D
:100200006428A50A3230AF004F2025080A3C0318A5
:100210000B290130A5002408033C03181029A40170
:10022000B72863000A148A100A118207BD28C4285F
:06023000CB28D028D528E0
:02400E00C431BB
:00000001FF
